 bc_example

 Timestamp is 4be8cfe0 (Tue May 11 12:32:48 2010)

 Preferred load address is 10000000

 Start         Length     Name                   Class
 0001:00000000 00000004H .CRT$XCA                CODE
 0001:00000004 00000004H .CRT$XCZ                CODE
 0001:00000008 00000004H .CRT$XIA                CODE
 0001:0000000c 00000004H .CRT$XIZ                CODE
 0001:00000010 00000004H .CRT$XPA                CODE
 0001:00000014 00000004H .CRT$XPZ                CODE
 0001:00000018 00000004H .CRT$XTA                CODE
 0001:0000001c 00000004H .CRT$XTZ                CODE
 0001:00000020 00000048H .rdata                  CODE
 0001:00000068 00000027H .rdata$debug            CODE
 0001:00000090 000011d0H .text                   CODE
 0001:00001260 00000018H .xdata                  CODE
 0001:00001278 00000028H .idata$2                CODE
 0001:000012a0 00000014H .idata$3                CODE
 0001:000012b4 0000005cH .idata$4                CODE
 0001:00001310 00000016H .idata$6                CODE
 0001:00001330 0000009eH .edata                  CODE
 0002:00000000 0000005cH .idata$5                DATA
 0002:0000005c 00000008H .data                   DATA
 0002:00000064 00000030H .bss                    DATA
 0003:00000000 00000168H .pdata                  DATA

  Address         Publics by Value              Rva+Base       Lib:Object

 0000:00000000       ___safe_se_handler_table   00000000     <absolute>
 0000:00000000       ___safe_se_handler_count   00000000     <absolute>
 0001:00000000       __xc_a                     10001000     corelib0:crt0init.obj
 0001:00000004       __xc_z                     10001004     corelib0:crt0init.obj
 0001:00000008       __xi_a                     10001008     corelib0:crt0init.obj
 0001:0000000c       __xi_z                     1000100c     corelib0:crt0init.obj
 0001:00000010       __xp_a                     10001010     corelib0:crt0init.obj
 0001:00000014       __xp_z                     10001014     corelib0:crt0init.obj
 0001:00000018       __xt_a                     10001018     corelib0:crt0init.obj
 0001:0000001c       __xt_z                     1000101c     corelib0:crt0init.obj
 0001:0000003c       ??_C@_0BI@INAEBFBK@PVRGetBufferClassJTable?$AA@ 1000103c     bufferclass_example.obj
 0001:00000054       ??_C@_1BE@KOOBJECM@?$AAs?$AAr?$AAv?$AAk?$AAm?$AA?4?$AAd?$AAl?$AAl?$AA?$AA@ 10001054     bufferclass_example_wince.obj
 0001:00000090       GetAnchorPtr               10001090 f   bufferclass_example.obj
 0001:000001b0       BC_Example_Register        100011b0 f   bufferclass_example.obj
 0001:000002e8       BC_Example_Unregister      100012e8 f   bufferclass_example.obj
 0001:00000374       BC_Example_Buffers_Create  10001374 f   bufferclass_example.obj
 0001:000004d4       BC_Example_Buffers_Destroy 100014d4 f   bufferclass_example.obj
 0001:00000580       BC_Example_Init            10001580 f   bufferclass_example.obj
 0001:00000594       BC_Example_Deinit          10001594 f   bufferclass_example.obj
 0001:000005a8       FillYUV420Image            100015a8 f   bufferclass_example_private.obj
 0001:000006d8       FillYUV422Image            100016d8 f   bufferclass_example_private.obj
 0001:00000800       FillRGB565Image            10001800 f   bufferclass_example_private.obj
 0001:000008f4       FillBuffer                 100018f4 f   bufferclass_example_private.obj
 0001:00000998       GetBufferCount             10001998 f   bufferclass_example_private.obj
 0001:000009bc       BCAllocKernelMem           100019bc f   bufferclass_example_wince.obj
 0001:000009c0       BCFreeKernelMem            100019c0 f   bufferclass_example_wince.obj
 0001:000009c4       BCAllocContigMemory        100019c4 f   bufferclass_example_wince.obj
 0001:00000a44       BCFreeContigMemory         10001a44 f   bufferclass_example_wince.obj
 0001:00000a70       CpuPAddrToSysPAddrBC       10001a70 f   bufferclass_example_wince.obj
 0001:00000a78       SysPAddrToCpuPAddrBC       10001a78 f   bufferclass_example_wince.obj
 0001:00000a80       BCOpenPVRServices          10001a80 f   bufferclass_example_wince.obj
 0001:00000aa8       BCClosePVRServices         10001aa8 f   bufferclass_example_wince.obj
 0001:00000ac0       BCGetLibFuncAddr           10001ac0 f   bufferclass_example_wince.obj
 0001:00000b74       OSPCIReadDword             10001b74 f   bufferclass_example_wince.obj
 0001:00000bc0       OSPCIWriteDword            10001bc0 f   bufferclass_example_wince.obj
 0001:00000c08       BCE_Init                   10001c08 f   bufferclass_example_wince.obj
 0001:00000ce4       BCE_Deinit                 10001ce4 f   bufferclass_example_wince.obj
 0001:00000d0c       BCE_Open                   10001d0c f   bufferclass_example_wince.obj
 0001:00000d10       BCE_Close                  10001d10 f   bufferclass_example_wince.obj
 0001:00000d18       BCE_IOControl              10001d18 f   bufferclass_example_wince.obj
 0001:00000d74       LoadLibraryW               10001d74 f   coredll:COREDLL.dll
 0001:00000d84       FreeLibrary                10001d84 f   coredll:COREDLL.dll
 0001:00000d94       GetProcAddressW            10001d94 f   coredll:COREDLL.dll
 0001:00000da4       MmMapIoSpace               10001da4 f   ceddk:CEDDK.dll
 0001:00000db4       MmUnmapIoSpace             10001db4 f   ceddk:CEDDK.dll
 0001:00000dc4       HalGetBusDataByOffset      10001dc4 f   ceddk:CEDDK.dll
 0001:00000dd4       HalSetBusDataByOffset      10001dd4 f   ceddk:CEDDK.dll
 0001:00000de4       DllMain                    10001de4 f   corelib0:dllmain.obj
 0001:00000f00       _DllMainCRTStartup         10001f00 f   corelib0:pegdmain.obj
 0001:00000f30       __GSHandlerCheckCommon     10001f30 f   corelib0:gshandler.obj
 0001:00000f6c       __GSHandlerCheck           10001f6c f   corelib0:gshandler.obj
 0001:00000f90       __security_init_cookie     10001f90 f   corelib0:seccinit.obj
 0001:00000fec       __security_check_cookie    10001fec f   corelib0:armsecgs.obj
 0001:00001000       __gsfailure                10002000 f   corelib0:armsecgs.obj
 0001:0000110c       _cexit                     1000210c f   corelib0:cexit.obj
 0001:00001128       _initterm                  10002128 f   corelib0:crt0dat.obj
 0001:0000115c       _cinit                     1000215c f   corelib0:crt0dat.obj
 0001:00001190       memcpy                     10002190 f   corelib1:COREDLL.dll
 0001:000011a0       malloc                     100021a0 f   corelib1:COREDLL.dll
 0001:000011b0       free                       100021b0 f   corelib1:COREDLL.dll
 0001:000011c0       mbstowcs                   100021c0 f   corelib1:COREDLL.dll
 0001:000011d0       strlen                     100021d0 f   corelib1:COREDLL.dll
 0001:000011e0       strcmp                     100021e0 f   corelib1:COREDLL.dll
 0001:000011f0       memset                     100021f0 f   corelib1:COREDLL.dll
 0001:00001200       _XcptFilter                10002200 f   corelib1:COREDLL.dll
 0001:00001210       __C_specific_handler       10002210 f   corelib1:COREDLL.dll
 0001:00001220       __security_gen_cookie2     10002220 f   corelib1:COREDLL.dll
 0001:00001230       __report_gsfailure         10002230 f   corelib1:COREDLL.dll
 0001:00001240       DisableThreadLibraryCalls  10002240 f   coredll:COREDLL.dll
 0001:00001250       TerminateProcess           10002250 f   coredll:COREDLL.dll
 0001:00001278       __IMPORT_DESCRIPTOR_COREDLL 10002278     coredll:COREDLL.dll
 0001:0000128c       __IMPORT_DESCRIPTOR_CEDDK  1000228c     ceddk:CEDDK.dll
 0001:000012a0       __NULL_IMPORT_DESCRIPTOR   100022a0     coredll:COREDLL.dll
 0002:00000000       __imp_MmMapIoSpace         10003000     ceddk:CEDDK.dll
 0002:00000004       __imp_HalSetBusDataByOffset 10003004     ceddk:CEDDK.dll
 0002:00000008       __imp_HalGetBusDataByOffset 10003008     ceddk:CEDDK.dll
 0002:0000000c       __imp_MmUnmapIoSpace       1000300c     ceddk:CEDDK.dll
 0002:00000010       \177CEDDK_NULL_THUNK_DATA  10003010     ceddk:CEDDK.dll
 0002:00000014       __imp_GetProcAddressW      10003014     coredll:COREDLL.dll
 0002:00000018       __imp_FreeLibrary          10003018     coredll:COREDLL.dll
 0002:0000001c       __imp_LoadLibraryW         1000301c     coredll:COREDLL.dll
 0002:00000020       __imp_memcpy               10003020     corelib1:COREDLL.dll
 0002:00000024       __imp___rt_udiv            10003024     corelib1:COREDLL.dll
 0002:00000028       __imp_malloc               10003028     corelib1:COREDLL.dll
 0002:0000002c       __imp_free                 1000302c     corelib1:COREDLL.dll
 0002:00000030       __imp_mbstowcs             10003030     corelib1:COREDLL.dll
 0002:00000034       __imp_strlen               10003034     corelib1:COREDLL.dll
 0002:00000038       __imp_strcmp               10003038     corelib1:COREDLL.dll
 0002:0000003c       __imp_memset               1000303c     corelib1:COREDLL.dll
 0002:00000040       __imp__XcptFilter          10003040     corelib1:COREDLL.dll
 0002:00000044       __imp___C_specific_handler 10003044     corelib1:COREDLL.dll
 0002:00000048       __imp___security_gen_cookie2 10003048     corelib1:COREDLL.dll
 0002:0000004c       __imp___report_gsfailure   1000304c     corelib1:COREDLL.dll
 0002:00000050       __imp_DisableThreadLibraryCalls 10003050     coredll:COREDLL.dll
 0002:00000054       __imp_TerminateProcess     10003054     coredll:COREDLL.dll
 0002:00000058       \177COREDLL_NULL_THUNK_DATA 10003058     coredll:COREDLL.dll
 0002:0000005c       __security_cookie          1000305c     corelib0:seccinit.obj
 0002:00000060       __security_cookie_complement 10003060     corelib0:seccinit.obj
 0002:00000078       gulDriverInitialised       10003078     bufferclass_example_wince.obj
 0002:0000007c       gulMemBase                 1000307c     bufferclass_example_wince.obj
 0002:00000080       gulMemCurrent              10003080     bufferclass_example_wince.obj
 0002:00000084       _exitflag                  10003084     corelib0:cexit.obj
 0002:00000088       __onexitend                10003088     <common>
 0002:0000008c       __onexitbegin              1000308c     <common>
 0002:00000090       _pRawDllMain               10003090     <common>

 entry point at        0001:00000f00

 Static symbols

 0001:000000a0       OpenBCDevice               100010a0 f   bufferclass_example.obj
 0001:000000bc       CloseBCDevice              100010bc f   bufferclass_example.obj
 0001:000000c4       GetBCBuffer                100010c4 f   bufferclass_example.obj
 0001:00000110       GetBCInfo                  10001110 f   bufferclass_example.obj
 0001:00000148       GetBCBufferAddr            10001148 f   bufferclass_example.obj
 0001:00000e04       _DllMainCRTStartupHelper   10001e04 f   corelib0:pegdmain.obj
 0001:00001044       doexit                     10002044 f   corelib0:cexit.obj
